:0600000010308600C92843
:100008009400030895000B118B100F1E43288F1DB9
:100018001A288F11061C3B28AE30810008308E004C
:10002800920115088300940E140E0900A630810071
:100038008E0803192A2806180310061C0314920CAC
:100048008E0315088300940E140E090006183B2829
:100058000408980016088400120880001808840014
:10006800960A40301602031D3B28193096008F016E
:100078008B120B1615088300940E140E09000F1628
:100088008F158B160B1220308B00EC308100150871
:100098008300940E140E0900C10A08304102031DA2
:1000A8005728C101C10A4108820761286E287B28A8
:1000B80088289528A228AF28BC28FF304102031DB4
:1000C8006D28C10A03304102031D6D28C1010130AA
:1000D80086065028FF304102031D7A28C10A0830DD
:1000E8004102031D7A28C101023086065028FF30DC
:1000F8004102031D8728C10A06304102031D8728D3
:10010800C101043086065028FF304102031D94289F
:10011800C10A0B304102031D9428C101083086062C
:100128005028FF304102031DA128C10A0C304102AA
:10013800031DA128C101103086065028FF30410256
:10014800031DAE28C10A04304102031DAE28C101B7
:10015800203086065028FF304102031DBB28C20A02
:1001680017304202031DBB28C201403086065028C2
:10017800FF304102031DC828C20A09304202031D8C
:10018800C828C2018030860650280930850006300C
:10019800650071306600093085001030860019301E
:1001A800960097008F0190308B00F1284022A130F3
:1001B800130203192329A23013020319402912300C
:1001C80013020319AB2B103013020319B12B14308F
:1001D80013020319A22BA623DA286400CD3062008B
:1001E80016081706031D85290519FD288518FF28F7
:1001F800F1288518F1288B138614402208308D00C9
:1002080006166130660006163A220A2906160310F9
:10021800900C031C122971306600152961306600A4
:1002280006163A228D0B0A29061671306600061644
:100238008F01E32186108B100B118B17F128C30156
:10024800C50140221308C400B723C20182238D23AD
:10025800FF306600A6237623883013020319382955
:10026800930140220616072808308C007623402286
:100278008C0B38290616072840221308C300402291
:100288001308C400C1234508930040224608930080
:100298004022421C522906164210072876231308CA
:1002A8008C0040228C0A762340228C0B5729061694
:1002B800072840221308C30040221308C400C123A2
:1002C800450893004022460893004022421C6F29AB
:1002D800061642100728762313088C0040228C0A41
:1002E8000C08C507031C7929C60A1D308C00762323
:1002F8004022C503031C8329C603031864298C0BF9
:100308007B29861405148515851C8629051D8629D3
:1003180008308D008B1317088400000891008B1794
:100328000310910C0318A3290510000005199A2938
:1003380005140000051D9E298D0B9429AD298511F2
:1003480000008518A52985150000851CA9298D0B95
:100358009429970A40301702031DB42919309700D1
:100368008610F12885018601063065007130660027
:10037800CC211222013041020319C729023041025F
:100388000319CA29BC290608E921BC291222BC295B
:100398000130650064000518CE296400051CD129C8
:1003A8001830C000C1010130EB2112224108C00001
:1003B8001222A5304102031DCC29A530E9290630B7
:1003C8008C0000008C0BE5290800C1000830C10032
:1003D800051064000B308100051CF0294008C0009E
:1003E8000000C00BF429C0000030C10C031C022A15
:1003F80065000130C00BFD296500092A6500013040
:10040800052A062AC00B032A6500C10BF2294008F9
:10041800C0000000C00B0D2A640008000830C100AD
:10042800051064000B308100051C182A4008C00024
:10043800003065000130C00B1E2A6500232A242ADB
:10044800252AC0010518262AC00A40084002051CB2
:10045800282AC10CC10B252A0518302A6400080077
:10046800003066000730C100C101860116308C00DB
:1004780000008C0B3C2A0800900108308D0085187C
:10048800512A051D432A85110310900C851C4A2A00
:10049800851500008D0B432A08000519432A05100D
:1004A8000314900C051D562A051400008D0B432AD1
:1004B80008000E34113411340A340434043404347A
:1004C80011341B34153411341134113411341134EE
:1004D800113411341134113411340E3404340C3401
:1004E80004340434043404340E340E341134013426
:1004F8000234043408341F340E3411340134063401
:1005080001340E340E341134013402340434083406
:100518001F340E34113401340634013411340E34CE
:10052800023406340A3412341F34023402341F34BD
:1005380010341E340134013411340E340E341134A5
:1005480001340634013411340E34023406340A34CA
:1005580012341F34023402341F3410341E34013470
:10056800013411340E340E34113410340E34113475
:1005780011340E341F34013401340234023404348B
:1005880004340E34113411340E34113411340E3451
:100598000E34113411340F34013411340E34003454
:1005A800003408340434023400340034023404348F
:1005B800083400340034003400340034003400348B
:1005C8000E34113411341F341134113411341F34E2
:1005D8001134113411341134113411340E341E34E1
:1005E800113411341134113411341E3411341134CE
:1005F8001E34113411341E341034103410341034B5
:10060800103410341F34103410341C3410341034A7
:100618001F34103410341C341034103410340134A6
:10062800013401340134013411340E3411341034DE
:100638001334113411340E34113413341134113489
:100648000E34113411341134153413340E34043487
:1006580004340E341134123414341834143412346B
:1006680011341B3415341134113411341134193444
:10067800153413341134113411340A340434043465
:10068800043411341B3415341134113411340A3440
:1006980004340434043411341B3415341134113443
:1006A800113411341934153413341134113411340C
:1006B8000A3404340434043407308C003C2A0430EF
:1006C8008C003C2A7E3430346D34793433345B34D6
:1006D8005F3470347F34733477341F344E343D3490
:1006E8004F34473486120000060893008616080027
:1006F8000611000013088600061508000030660081
:100708002D308600061142088600000006150610E6
:10071800080086140611000043088600061500002C
:1007280006110000440886000615000006110000A6
:1007380045088600061500008610080040221308A8
:10074800860007288617061FA72B86130800003087
:1007580066004022130886000728FF306600060856
:10076800930040220728C40DC40DC50DC40DC50D46
:10077800C40DC50D0F30C40508000430C300C50101
:100788004308C400B72344088C0006160000C201C1
:1007980082238D23FF306600A62342107623FE3085
:1007A80013020319DB2B4214C501C6010800762386
:1007B8001308C5001308C30076231308C6001308DE
:1007C800C4008C038C080319FE2B2030C307031CBC
:1007D800F12BC40A031CF12BC50AC408031DF82B0E
:1007E80020304302031CC92B2030C302031CE92B11
:0607F800C403E92B080018
:1042000000000000000000000000000000000000AE
:10421000000000000000000000000000000000009E
:10422000000000000000000000000000000000008E
:10423000000000000000000000000000000000007E
:10424000000000000000000000000000000000006E
:10425000000000000000000000000000000000005E
:10426000000000000000000000000000000000004E
:10427000000000000000000000000000000000003E
:084000007F007F007F007F00BC
:02400E00F53F7C
:02FFFE00840F6E
:00000001FF
